:1000000083168510051005118511831285140510BE
:1000100008308C000530900003309008031D8506E1
:100020000F30000000008D1F103E3E20033090086E
:10003000031D8506000005150D308D1F103E8D0D2A
:100040008C0B3C288E0008308C0006088D008F0633
:10005000031D3228900803193728900B3728851183
:1000600085103728851505309000851400000D088F
:100070008F0005110E08FA3E3E200C288E008E0BD4
:040080003F2808000D
:084000000000000001000300B4
:02400E00F23F7F
:00000001FF
